:103F0F000F580F4E0F430F380F2D0F210F140F07A0
:103F1F000EF90EEB0EDC0ECC0EBC0EAB0E9A0E870E
:103F2F000E750E610E4D0E380E220E0C0DF40DDCBB
:103F3F000DC40DAA0D900D750D5A0D3E0D210D03DB
:103F4F000CE40CC50CA50C850C640C420C200BFD6D
:103F5F000BD90BB50B900B6B0B460B200AF90AD341
:103F6F000AAC0A840A5D0A350A0D09E409BC0993F3
:103F7F00096B0942091A08F108C808A00878085007
:103F8F000828080007D807B1078A0764073E0718F3
:103F9F0006F206CD06A906840661063E061B05F845
:103FAF0005D705B50595057405550535051704F9AC
:103FBF0004DB04BE04A20486046A044F0435041B08
:103FCF00040203E903D103B903A2038B0375035F53
:103FDF00034A03350321030D02FA02E702D502C398
:103FEF0002B102A0028F027F026F025F02500241F4
:103FFF00023302250217020A01FD01F001E301D786
:10400F0001CC01C001B501AA019F0195018B01816E
:10401F000178016E0165015C0154014B0143013BC5
:10402F000133012C0125011D0116011001090102A7
:10403F0000FC00F600F000EA00E500DF00DA00D433
:10404F0000CF00CA00C600C100BC00B800B300AF6B
:10405F0000AB00A700A3009F009B00980094009165
:10406F00008D008A00870084008100010C0101058A
:10407F0002011E030A9604013205030306006407BA
:10408F00010108000009015A0E01010F0001120081
:10409F006413010114013C1501FA1664FA17FFFFAE
:1040AF001D00072000072400022701012F013C30CB
:1040BF00020232010335FFFF3603073CFFFF3DFFCE
:1040CF00FF180002191E461A00021B00022D32C8EB
:0640DF002E0001FAFAFABE
:10004800900786E0FEA3E0FF7457BE0010D39F40E0
:100058000C90407912001EE493F59980129007865F
:10006800E0FEA3E0FF90407912001EE493F599901A
:10007800078612000E900786E0FEA3E0FF746C6FFF
:100088004E700375130022900072E0B402087401E8
:10009800900072F0D20F90013AE090002AF090019F
:1000A8003BE090002BF090013CE090002CF0A20A7D
:1000B800B3401690013AE0700C90013BE070069056
:1000C800013CE060028002C20A90013AE0B4300FBD
:1000D80090013BE0B4470890013CE0643B6002803B
:1000E80004D20B8002C20BE559B40102800302025C
:1000F80011900057E0F567900062E0F569900063A1
:10010800E0F56A900074E0F56B90007AE0900029C1
:10011800F090007CE0F56690007DE0F56890008046
:10012800E0F565900081E0F564900090E090004172
:10013800F0900091E0900042F0900092E09000432F
:10014800F0900093E0900044F0900094E090004517
:10015800F0900095E0900046F0900096E0900047FF
:10016800F0900097E0900048F0900099E0900033FC
:10017800F090009AE0900034F090009BE0900035F9
:10018800F090009CE0900036F0900079E0B4011700
:1001980090000A740FF0A374FFF090000CE4F0A331
:1001A800F07402900079F0900079E0B4035990005F
:1001B8000CE0FEA3E0FF90000AE0FCA3E0FD1200C3
:1001C8000374101242457408124237EF900026F06B
:1001D800EF700674FF900026F07400900079F0909C
:1001E800000BE0900027F090000AE0900028F090C3
:1001F8000026E0900789F0900027E090078AF090A9
:100208000028E090078BF0803F900081E070067531
:100218005901756400A20AB3402E90013AE090009B
:100228002AF090013BE090002BF090013CE0900018
:100238002CF090002AE0700C90002BE070069000E3
:100248002CE060028002C20AE5677003756702E568
:100258006970037569027E837FC2E5678E048F0526
:10026800FF1242278C398D3AE56A75F0FAA4FFAE81
:10027800F0E5698E048F05FF1242278C3D8D3E9074
:10028800004FE0F56190004DE0FE900069E0B50692
:100298001890004CE0FE900068E0B5060C90004B0A
:1002A800E0FE900059E06E606F900069E070069083
:1002B8000068E060067400900059F0900069E0B4AE
:1002C80002089000497401F08005900049E4F0901C
:1002D8000068E0B4020890004A7401F080059000BC
:1002E8004AE4F0900068E0600690004AE06002800E
:1002F800057561048003756105E55AB55902D20F89
:10030800900068E090004CF0900069E090004DF09B
:10031800900059E090004BF0740190009EF074003A
:1003280090009FF074019000A0F074009000A1F07C
:1003380074019000A2F074009000A3F07400900083
:10034800A4F074009000A5F074019000A6F0740069
:100358009000A7F074019000A8F074019000A9F033
:1003680074019000AAF074009000ABF07401900042
:10037800ACF074009000ADF074019000AEF0740021
:100388009000AFF074019000B0F074009000B1F0EC
:1003980074009000B2F07401900362F0740090034E
:1003A80063F07400900364F07401900365F07401C5
:1003B800900366F07401900367F07400900368F08E
:1003C80074019003A2F074019003A3F074009003E9
:1003D800A4F074009003A5F074019003A6F07401D2
:1003E8009003A7F074009003A8F074009003E2F063
:1003F80074019003E3F074009003E4F07400900338
:10040800E5F074019003E6F074009003E7F07400DF
:100418009003E8F07400900422F07401900423F033
:100428007400900424F07400900425F07400900483
:1004380026F07400900427F07400900428F07400EB
:10044800900462F07400900463F07400900464F007
:100458007400900465F07400900466F074009004D1
:1004680067F07400900468F022E5B554F7F5B5C25A
:10047800A1C293C294C291C292757000E5B554FDB1
:10048800F5B5C207E5B554FBF5B5755105E5510459
:10049800F55290004FE0F561900025E4F0C209E5BF
:1004A800B554FEF5B5C28E758D00758B00754C0080
:1004B800752600752500D28E22750A00750900AED2
:1004C80009AF0A7457BE00039F500302057E90408F
:1004D8007912001EE49390004E12425D0FBF000196
:1004E8000EE0FC90407912001EECFEE493FFEEC390
:1004F8009F5026AE09AF0A0FBF00010E9040791237
:10050800001EAE09AF0AE493FC90407912001EE485
:100518009390004E12425DECF0AE09AF0A9040791C
:1005280012001EE49390004E12425DE0FC90407B66
:1005380012001EECFCE493FDECD39D401990407B27
:1005480012001EE493FC90407912001EE493900080
:100558004E12425DECF0AE09AF0A74022FFF500153
:100568000E8E098F0A780A740126F6500418E436AC
:10057800F640030204C722750A00750900AE09AFE8
:100588000A7415BE00039F500302064C9040D01217
:10059800001EE49390004E12425D0FBF00010EE072
:1005A800FC9040D012001EECFEE493FFEEC39F5077
:1005B80026AE09AF0A0FBF00010E9040D012001EF0
:1005C800AE09AF0AE493FC9040D012001EE4939069
:1005D800004E12425DECF0AE09AF0A9040D0120016
:1005E8001EE49390004E12425DE0FC9040D212004F
:1005F8001EECFCE493FDECD39D40199040D2120010
:100608001EE493FC9040D012001EE49390004E121A
:10061800425DECF0AE09AF0A740F6F4E7006750AB2
:1006280015750900AE09AF0A74022FFF50010E8E2E
:10063800098F0A780A740126F6500418E436F64041
:100648000302058522054D22054C22054EC2CF2204
:1006580090F800E4936406600280FE75840175A733
:100668000075FF80900788E4F075C91075A70F75AD
:10067800A1C775A70075D90075CEFF75A70F75F1CD
:10068800FE75F2FF75F33775F47875A4BA75A5FF92
:1006980075A60775AE0075AFFF75D48175D5FF7562
:1006A800D6FF75D7FFE5B554EFF5B5E5B554DFF5D9
:1006B800B5C287E5B554BFF5B5E5B5547FF5B57551
:1006C800A70075A20175A14775F80975BC0175BE2B
:1006D8000475BD6C75BE0775BDA075BE0875BD01F6
:1006E80075BC0075BB1875BC2075BA0875E88075AF
:1006F800D11375A70F75E10575E20075C7407597A9
:1007080000759780740A1242177597C0E5975420B0
:10071800700280F8758F0275A700D2AF75980075C2
:10072800A90C75A70F75AB4375ADFB75AC1E75A706
:1007380000758911758E00758C00758A00D2A9D252
:100748008C758D00758B00D2ABD28E75CD0075CCB3
:100758000075CA0075CB00D2ADC2CFD2CA7591045C
:100768007592007593CD75EF0675D94075CF0190D8
:100778000786E4F0A3F0751300751400C299D20A35
:10078800C21012047174C8F51875170012283E7546
:10079800A70FE5FB90001AF0E5FA90001BF0E5F9C9
:1007A80090001CF075A70090F800E493F508122952
:1007B80075122EAF900789E0900026F090078AE026
:1007C800900027F090078BE0900028F090078CE0CD
:1007D800900029F090078DE0F56790078EE0F569A5
:1007E80090078FE0F56A900790E0F56B900791E02D
:1007F800F566900792E0F568900793E0F565900735
:1008080094E0F564900795E090002AF0900796E050
:1008180090002BF0900797E090002CF0900798E05C
:10082800900041F0900799E0900042F090079AE01C
:10083800900043F090079BE0900044F090079CE004
:10084800900045F090079DE0900046F090079EE0EC
:10085800900047F090079FE0900048F09007A0E0D4
:10086800900033F09007A1E0900034F09007A2E0E8
:10087800900035F09007A3E0900036F074009000E7
:1008880082F090013AE0700C90013BE07006900114
:100898003CE060028004C20A8002D20A90F807E4B1
:1008A80093900021F0900021E0440A900021F090FC
:1008B8000021E054FE900021F07406900012F074BC
:1008C80002900013F090F802E493900014F074037F
:1008D800900015F07403900016F0741E900017F045
:1008E8007405900018F07405900019F090F804E46D
:1008F8009390001DF0740090001EF090F805E493AA
:1009080090001FF090F806E493900020F074FF9098
:100918000022F0745A900125F07446900126F07474
:1009280020900127F07435900128F074489001292F
:10093800F0745090012AF0743290012BF0743490C6
:10094800012CF0742090012DF0743590012EF07474
:100958005390012FF07470900130F074659001315C
:10096800F07465900132F07464900133F090007A6D
:10097800E0D394014006740090007AF0755901752F
:100988005A01740390004CF012008F1204C1120532
:100998007F12286AE5B554FEF5B5900025E4F0907D
:1009A8000786E4F0A3F075240075230075480075E8
:1009B8002A00752900754900753200753100754A9D
:1009C80000755400755500755B0075510575520129
:1009D80075343C7533007572007571007573CD758B
:1009E80056007557007558007543007544007545E5
:1009F80000754600755C007547007542007541003A
:100A0800900006E4F0A3F0900008E4F0A3F0755F0E
:100A18000075600090000E74FDF0A374E8F090007B
:100A280023E4F07464900024F0C200D201C202D220
:100A380003754D00756E00C297C2A0C296C295C2DA
:100A4800A2C20F7E017F00900028E012424590006C
:100A580027E02FFF50010E90000AEEF0A3EFF09070
:100A68000026E0700674FF900026F090000AE0FE71
:100A7800A3E0FFEFD394FFEE940F400790000AE441
:100A8800F0A3F07400900071F07400900079F07495
:100A980000900082F0740090008DF074009000B413
:100AA800F0E5687003756804743A90074EF074FDB9
:100AB80090074FF0900414E0900454F0D2B0D2B7ED
:100AC800D2A7D2A6D2B1D2A3C207A2B6B39204A229
:100AD800B3B39205D29CD2EC75CF01A298B340056E
:100AE800C298123213E5136006A299B3B34002808C
:100AF80005C299123783E51464016005E514B4044E
:100B08000280D5E54DD39405400CE55BC394C850ED
:100B180002055B754D00E573C394F0501A787112A5
:100B2800003FAE71AF72EFD394E8EE94034008052E
:100B380073757200757100C28E7E047F00E54C12D9
:100B48004245E58D75F004A4FDACF0EF2DFDEE3CBB
:100B5800FCE58B75F04084FF7E00ED2FFFEC3EFE38
:100B68008E258F26D28EA2B6300401B35003020C14
:100B7800A7A2B6300401B35003020CA7A2B640677F
:100B88000554A210400575FFA0D210E5B54401F543
:100B9800B5900024E4F0E554D3956740487C837D04
:100BA800C2AE25AF261240E58E238F24E5482FFFDD
:100BB80050010E74011242378E238F248524487504
:100BC8005401C28E758D00758B00754C00D28E74E1
:100BD80003BE00039F50069000257401F0E543B45E
:100BE8000603754300D204A2B6B35003020CA7C291
:100BF8000490006BE060181238C4A200B34008E506
:100C0800B54408F5B58006E5B554F7F5B58002C2D8
:100C18000090006EE06010123A19A202B34004D2AC
:100C2800A18002C2A18002C2A1A207B34004D29649
:100C38008002C296900059E06004D2958002C29565
:100C480090004AE0B40104D2978002C2979000490C
:100C5800E0B40104D2A08002C2A0A209B34004D229
:100C6800A28002C2A2900018E0FE900014E0C39E89
:100C78004009900014E0D39408400974FB900023C5
:100C8800F012047190001DE0601590001DE0FE90C8
:100C98000017E06E600974FE900023F0120471C220
:100CA800CA7E017F00E54E124245E5CD2FFF500177
:100CB8000E8E278F28D2CAE566B4014890000EE050
:100CC800FCA3E0FDEFC39DEE9C4039B208E52A4540
:100CD800296013A208B34008E5B54404F5B58006B9
:100CE800E5B554FBF5B590000EE0FEA3E0FF9000DB
:100CF80010E0FCA3E0FDEF2DFDEE3CFC90000EECB7
:100D0800F0A3EDF0A2B3300501B35003020DF5A234
:100D1800B3300501B35003020DF5A2B35003020D21
:100D2800EE0555A210400575FFA0D210E5B54401A7
:100D3800F5B5900024E4F0E555D395695003020D0C
:100D4800EC7CEA7D60AE27AF281240E58E298F2A19
:100D5800E56A12424574FF8E048F05FF1242278C04
:100D6800298D2AE5492DFD50010C74018C068D074B
:100D78001242378E298F2A852A49A209B340157451
:100D880064124245900067E08E048F05FF124227E7
:100D98008C298D2A75550190000EE0FEA3E0FFAC6A
:100DA80027AD2812000390000EEEF0A3EFF0E568DF
:100DB800FF124227740AFF12422790007BE08C063C
:100DC8008D0712424574148E048F05FF1242279036
:100DD8000010ECF0A3EDF0C2CA75CD0075CC00751B
:100DE8004E00D2CAD205A2B3B34002C20590002574
:100DF800E0B40107E556C39406400302140DE56EFE
:100E080090281DF8282873900059E0C394024003E5
:100E1800020F63E551D394015003020F63E5517546
:100E2800F040A4FFAEF090031212001EE0C39545F7
:100E38005018E55175F040A4FFAEF0900311120070
:100E48001EE0F52E752D00020F63E55175F040A4E4
:100E5800FFAEF090031012001EE0C3954540030258
:100E68000EFFE55175F040A4FFAEF090031112009B
:100E78001EE55175F040A4FFAEF0E0FC90030F12A0
:100E8800001EECFEE0FFEEC39FFEE5518E0475F0F8
:100E980040A4FFAEF090031012001EE0F4042545B4
:100EA8008C0088F0A4FFAEF0E5518F048E0575F034
:100EB80040A4FFAEF090031212001EE55175F040F9
:100EC800A4FFAEF0E0FA90031012001EEAFEE0FF65
:100ED800EEC39FFECDCCCD8E07124227E55175F0AB
:100EE80040A4FFAEF090030F12001EE02DFD50014C
:100EF8000C8C2D8D2E8064E55175F040A4FFAEF06A
:100F080090030F12001EE55175F040A4FFAEF0E00B
:100F1800FC90030E12001EECFEE0FFEEC39F854519
:100F2800F0A4FFAEF0E5518F048E0575F040A4FFE4
:100F3800AEF090031012001EE0FECDCCCD8E07124D
:100F48004227E55175F040A4FFAEF090030E120061
:100F58001EE02DFD50010C8C2D8D2E756E01021496
:100F68000D900059E0C39402400302111790004FFE
:100F7800E0D3955150030210BFE55175F040A4FF2E
:100F8800AEF090031812001EE0C395455018E551C5
:100F980075F040A4FFAEF090031712001EE0F52C88
:100FA800752B000210BFE55175F040A4FFAEF0901C
:100FB800031612001EE0C39545400302105BE5517D
:100FC80075F040A4FFAEF090031712001EE55175AE
:100FD800F040A4FFAEF0E0FC90031512001EECFEFA
:100FE800E0FFEEC39FFEE5518E0475F040A4FFAE0E
:100FF800F090031612001EE0F40425458C0088F0DA
:10100800A4FFAEF0E5518F048E0575F040A4FFAE45
:10101800F090031812001EE55175F040A4FFAEF0E1
:10102800E0FA90031612001EEAFEE0FFEEC39FFEF0
:10103800CDCCCD8E07124227E55175F040A4FFAE06
:10104800F090031512001EE02DFD50010C8C2B8D25
:101058002C8064E55175F040A4FFAEF090031512A2
:10106800001EE55175F040A4FFAEF0E0FC900314BB
:1010780012001EECFEE0FFEEC39F8545F0A4FFAE14
:10108800F0E5518F048E0575F040A4FFAEF0900393
:101098001612001EE0FECDCCCD8E07124227E55178
:1010A80075F040A4FFAEF090031412001EE02DFD71
:1010B80050010C8C2B8D2CE551B40123E561D394A0
:1010C80001401CE55604D395514014E545C39405E9
:1010D800500D90035FE0A829B80006952A400280C9
:1010E80003755102E551B5612290004FE0D3955147
:1010F8004019E55175F040A4FFAEF09003171200B7
:101108001EE0A823B80006952440028002056175F8
:101118006E0202140D900059E0B4022AE55175F0F0
:1011280040A4FFAEF090031712001EE0F52C752BBB
:1011380000E55175F040A4FFAEF090030E12001EBA
:10114800E0F52E752D00900059E0B4030F90005182
:10115800E0F52C752B00752E00752D00756E0302B9
:10116800140DE55175F040A4FFAEF0900320120075
:101178001EE0C3955B4003021243900049E07036BD
:10118800E551D394014029AE23AF24AC2DAD2EED0B
:10119800D39FEC9E401AE55175F040A4FFAEF09045
:1011A800031E12001EE0A829B80005D3952A500294
:1011B800800215518034E551D394024029AE23AF03
:1011C80024AC2DAD2EEDD39FEC9E401AE55175F061
:1011D80040A4FFAEF090031E12001EE0A829B8003C
:1011E80005D3952A500280021551E551B55237E5CD
:1011F80051C395615030E55604D395514028AE232C
:10120800AF24AC2BAD2CEFD39DEE9C4019E5517566
:10121800F040A4FFAEF090031F12001EE0A829B80A
:101228000006952A400280020551E5B554FDF5B542
:10123800E55165526005C207755B00756E040214BE
:101248000DE55175F040A4FFAEF090031A12001E90
:10125800E0B40117E55175F040A4FFAEF09003200B
:1012680012001EE0240AC3955B400302131975306F
:1012780064752F00A207B3500B900060E02405C3EB
:1012880095454003021319E55175F040A4FFAEF0EF
:1012980090031D12001EE0C395454064E55175F0AA
:1012A80040A4FFAEF090031C12001EE55175F040FB
:1012B800A4FFAEF0E0FC90031B12001EECFEE0FF62
:1012C800EEC39F8545F0A4FFAEF0E5518F048E056F
:1012D80075F040A4FFAEF090031D12001EE0FECD95
:1012E800CCCD8E07124227E55175F040A4FFAEF031
:1012F80090031B12001EE02DFD50010C8C2F8D3029
:10130800AE23AF24AC2FAD30EFD39DEE9C4002D27C
:1013180007756E0502140DE551B40109900059E0F6
:10132800C3940240030213ED900358E0D39545504F
:10133800030213ED900356E0C395455040900357C0
:10134800E0FE900355E0F4042EFE900356E0F4040A
:1013580025458E0088F0A4FFAEF0900358E0FC907D
:101368000356E0F4042C8E048F05FF1242279003E5
:1013780055E02DFD50010C8C2B8D2C802C900355A5
:10138800E0FE900354E0F4042E8545F0A4FFAEF08F
:10139800900356E08E048F05FF124227900354E015
:1013A8002DFD50010C8C2B8D2CE551C395615030CF
:1013B800E55604D395514028AE23AF24AC2BAD2C71
:1013C800EFD39DEE9C4019E55175F040A4FFAEF0B7
:1013D80090031F12001EE0A829B80006952A4002B3
:1013E8008003755102900049E0B40106E55164019B
:1013F80060028003755102E55165526005C20775A8
:051408005B00756E00A1
:10281D00020E0F020F6902111D02116A0212490206
:02282D00131F77
:10140D00900050E02402A823B80007D39524400291
:10141D00C207900025E0B40109900059E0C3940380
:10142D004003021595900049E060030214E4E55174
:10143D00D394014034E55175F040A4FFAEF0900314
:10144D001412001EE0A823B8001FD39524401AE5FE
:10145D005175F040A4FFAEF090031F12001EE0A8DE
:10146D0029B80005D3952A500280021551E551D3B4
:10147D009401402FE55175F040A4FFAEF09003129A
:10148D0012001EE0C39545501AE55175F040A4FFBA
:10149D00AEF090031E12001EE0A829B80005D395EA
:1014AD002A500280021551E551D394014022E55690
:1014BD0004C39551501AE55175F040A4FFAEF0905C
:1014CD00031E12001EE0A829B80005D3952A50026C
:1014DD008002155102158AE551D394024034E5512D
:1014ED0075F040A4FFAEF090031412001EE0A82387
:1014FD00B8001FD39524401AE55175F040A4FFAEF6
:10150D00F090031F12001EE0A829B80005D3952AFC
:10151D00500280021551E551D39402402FE55175CB
:10152D00F040A4FFAEF090031212001EE0C39545EB
:10153D00501AE55175F040A4FFAEF090031E120055
:10154D001EE0A829B80005D3952A50028002155136
:10155D00E551D394024022E55604C39551501AE546
:10156D005175F040A4FFAEF090031E12001EE0A8CE
:10157D0029B80005D3952A500280021551E5516511
:10158D00526005C207755B00900060E0D395455031
:10159D0009900054E0C395455002C207900059E0F0
:1015AD0070030217FAA2A5B34008A2A4B340030228
:1015BD0017E3AE35AF367441D39F749C9E400578CA
:1015CD003512003FAE35AF36EFB48806EEB41302D8
:1015DD0080030217C0A2A55003021683900059E0A4
:1015ED00B4010B90004FE0D395614002056190006E
:1015FD0059E0B40254E55175F040A4FFAEF09003EC
:10160D002012001EE0C3955B503F90004FE0D39534
:10161D00514021E55604D395514019E55175F040DF
:10162D00A4FFAEF090031412001EE0A823B800062C
:10163D00952440028002055190004FE0F561E5517F
:10164D0065526005C207755B00900059E0B4032632
:10165D0090004FE0D395514008E55604D395515075
:10166D00028002055190004FE0F561E55165526031
:10167D0005C207755B00A2A450030217C090005964
:10168D00E0B4016E900049E07035E551D39401400E
:10169D0029E55175F040A4FFAEF090031E12001E17
:1016AD00E0A829B8000FD3952A400A1551755B00A3
:1016BD00855161800385516180037561018033E53A
:1016CD0051D394024029E55175F040A4FFAEF0903E
:1016DD00031E12001EE0A829B8000FD3952A400A58
:1016ED001551755B008551618003855161800375CE
:1016FD006102900059E0D3940150030217B4E551F3
:10170D0075F040A4FFAEF090032012001EE0C395CB
:10171D005B40030217B4900049E07041E551D3944A
:10172D00014034E55175F040A4FFAEF09003111265
:10173D00001EE0A823B8001FD39524401AE551756B
:10174D00F040A4FFAEF090031E12001EE0A829B8D1
:10175D000005D3952A500280021551803FE551D3E3
:10176D0094024034E55175F040A4FFAEF0900311A2
:10177D0012001EE0A823B8001FD39524401AE5518E
:10178D0075F040A4FFAEF090031E12001EE0A829D4
:10179D00B80005D3952A500280021551E5516552C6
:1017AD006005C207755B00E556B40704055F80034D
:1017BD00755F00E564B4010EAE35AF36EF64407071
:1017CD0005EE649C6002800EA2A54003755901A22E
:1017DD00A44003755902A2A5B3B35006A2A4B3B396
:1017ED00400280067536007535000218E8A2A5B3D3
:1017FD004008A2A4B340030218D4AE35AF367441ED
:10180D00D39F749C9E4005783512003FAE35AF36A0
:10181D00EFB48806EEB4130280030218D4A2A540DB
:10182D006F900068E0605A90004AE0B401079000A4
:10183D004AE4F0800690004A7401F090004AE0708E
:10184D0005756104800375610590004AE0B40104DB
:10185D00D2978002C297E551B4051AE55175F04053
:10186D00A4FFAEF090031E12001EE0A829B80005DB
:10187D00D3952A50028008755104C207755B00800C
:10188D0003756105E556B40704055F8003755F00B8
:10189D00A2A44033900069E06021900049E0B401BA
:1018AD0007900049E4F080069000497401F0900023
:1018BD0049E0B40104D2A08002C2A0E556B40704E9
:1018CD00055F8003755F00A2A5B3B35006A2A4B354
:1018DD00B340028006753600753500E559655A60CE
:1018ED0006900082E06003021A70C29C75140075A8
:1018FD001300C2CAE55990282FF8282873801212B8
:10190D002EAF800D122F88800812306180031231A6
:01191D003A8F
:0F282F0002190A02190C02191102191602191BBB
:10191E00900029E090007AF0E567900057F0E569B5
:10192E00900062F0E56A900063F0E56B900074F051
:10193E00E56690007CF0E56890007DF0E56590002E
:10194E0080F0E564900081F090002AE090013AF07A
:10195E0090002BE090013BF090002CE090013CF0C9
:10196E00900041E0900090F0900042E0900091F0E5
:10197E00900043E0900092F0900044E0900093F0CD
:10198E00900045E0900094F0900046E0900095F0B5
:10199E00900047E0900096F0900048E0900097F09D
:1019AE00900033E0900099F0900034E090009AF0AF
:1019BE00900035E090009BF0900036E090009CF097
:1019CE007400900082F0745A900125F074469001D4
:1019DE0026F07420900127F07435900128F0744899
:1019EE00900129F0745090012AF0743290012BF07E
:1019FE00743490012CF0742090012DF07435900108
:101A0E002EF0745390012FF07470900130F07465C5
:101A1E00900131F07465900132F07464900133F0EE
:101A2E009003D4E0900414F0743A90074EF074FDD5
:101A3E0090074FF012008F900004E4F0A3F0900096
:101A4E00067475F0A37430F09000087475F0A374EA
:101A5E0030F085595AD2CA754C00D29C741B900036
:101A6E0023F0900025E0B401028003021ECFE5565C
:101A7E00C394065005E551B55203021B5FC207E53C
:101A8E005175F040A4FFAEF090032212001EE0301C
:101A9E00E003D38001C3B34008E5B54410F5B5802B
:101AAE0006E5B554EFF5B5E55175F040A4FFAEF07F
:101ABE0090032312001EE030E003D38001C3B34035
:101ACE0008E5B54420F5B58006E5B554DFF5B5E576
:101ADE005175F040A4FFAEF090032412001EE030CA
:101AEE00E003D38001C39287E55175F040A4FFAEA9
:101AFE00F090032512001EE030E003D38001C39264
:101B0E000CE55175F040A4FFAEF090032612001EB6
:101B1E00E030E003D38001C3920DE55175F040A48F
:101B2E00FFAEF090032712001EE030E003D38001D9
:101B3E00C3920E855152AE29AF2A7405BE00039F83
:101B4E005007E545D3940550028006E5B54402F5ED
:101B5E00B5E556D394055003021DCEC207E551D309
:101B6E0094015003021C62E55175F040A4FFAEF0E3
:101B7E0090031E12001EE0A829B80007D3952A4034
:101B8E00021551E55165527003021C5FE55175F067
:101B9E0040A4FFAEF090032212001EE030E003D30B
:101BAE008001C3B34008E5B54410F5B58006E5B530
:101BBE0054EFF5B5E55175F040A4FFAEF090032358
:101BCE0012001EE030E003D38001C3B34008E5B538
:101BDE004420F5B58006E5B554DFF5B5E55175F051
:101BEE0040A4FFAEF090032412001EE030E003D3B9
:101BFE008001C39287AE29AF2A7405BE00039F50A1
:101C0E0002D287E55175F040A4FFAEF09003251285
:101C1E00001EE030E003D38001C3920CE55175F055
:101C2E0040A4FFAEF090032612001EE030E003D376
:101C3E008001C3920DE55175F040A4FFAEF0900304
:101C4E002712001EE030E003D38001C3920E8551AF
:101C5E0052021DCEE556B406709000ACE030E0089E
:101C6E00E5B54410F5B58006E5B554EFF5B5900031
:101C7E00ADE030E008E5B54420F5B58006E5B55495
:101C8E00DFF5B59000AEE030E003D38001C392875C
:101C9E009000AFE030E003D38001C3920CE55BD33C
:101CAE0094034002D20C9000B0E030E003D38001E8
:101CBE00C3920D9000B1E030E003D38001C3920EC9
:101CCE00E55BD394034002D20EE556B4077D900037
:101CDE00A5E030E008E5B54410F5B58006E5B5544D
:101CEE00EFF5B59000A6E030E008E5B54420F5B577
:101CFE008006E5B554DFF5B5AE29AF2A7406BE00F1
:101D0E0011D39F400D9000A7E030E003D38001C3B4
:101D1E0092879000A8E030E003D38001C3920CE5D7
:101D2E005BD394034002C20C9000A9E030E003D3D1
:101D3E008001C3920D9000AAE030E003D38001C36E
:101D4E00920EE55BD394034002C20EE556B40870C2
:101D5E0090009EE030E008E5B54410F5B58006E54C
:101D6E00B554EFF5B590009FE030E008E5B544209E
:101D7E00F5B58006E5B554DFF5B59000A0E030E08E
:101D8E0003D38001C392879000A1E030E003D3809B
:101D9E0001C3920CE55BD394034002D20C9000A2D7
:101DAE00E030E003D38001C3920D9000A3E030E059
:101DBE0003D38001C3920EE55BD394034002D20E8F
:101DCE00E551B40107E556C3940640028012E55B67
:101DDE00D394034002C20CE55BD394034002C20EBF
:101DEE00900072E06058E54575F00284FF7E009029
:101DFE00014E12001EE0F55DE54775F00A84FF7E88
:101E0E000090024E12001EE0F55EE55D255ED39455
:101E1E0064400BE55D255EC39464F55D8003755DDE
:101E2E0000E55D75F00284FF7E008F5DEFC3943395
:101E3E005007EF24CDF55D8003755DFF801CE545F1
:101E4E0075F00284FF7E0090014E12001EE075F0C8
:101E5E000284FF7E00EF24CDF55DE595C3955D40D0
:101E6E0004C2938002D293A207B34005E556B4078D
:101E7E00037573CDE595C395734004C2948002D269
:101E8E0094E54575F00284FF7E0090018012001EDD
:101E9E00E075F00284FF7E00EF24CDF570E595C36A
:101EAE0095705017A20CB34002D291A20DB340020E
:101EBE00D292A20EB34002D2908006C291C292C2BA
:101ECE0090E543C39406400302253AA2EDB35003B6
:101EDE0002253AC2EDE54360030220347E017F0005
:101EEE00E5BE124245E5BD2FFF50010E900000EEFB
:101EFE00F0A3EFF0900029E0B401177E0F7FFF9062
:101F0E000000E0FCA3E0FD120003900000EEF0A341
:101F1E00EFF0900079E0B4025B900000E0FEA3E0E9
:101F2E00FF90000AE0FCA3E0FDEDD39FEC9E400F76
:101F3E00900000E0F8A3E090000AC8F0A3C8F0906B
:101F4E000000E0FEA3E0FF90000CE0FCA3E0FDEF3C
:101F5E00D39DEE9C400F900000E0F8A3E090000CA3
:101F6E00C8F0A3C8F0900000E0FEA3E0FF740412D6
:101F7E0042378F44900079E07060900000E0FEA33D
:101F8E00E0FF90000AE0FCA3E0FDEFD39DEE9C4045
:101F9E000D120003900000EEF0A3EFF0800790000A
:101FAE0000E4F0A3F0900000E0FEA3E0FF74101236
:101FBE004245900026E08E048F05FF1242279000C6
:101FCE0000ECF0A3EDF07400D39D74019C400890DA
:101FDE000001E0F54480037544FFE54475F00AA462
:101FEE00FFAEF074198E048F05FF1242278D45ED5A
:101FFE002532FFAE3150010E74011242378F4585E6
:10200E004532753100EFD3946240037545629000FE
:10201E0072E064016006900066E060028005754320
:10202E0001800375BB17E543B4010280030221242E
:10203E007E017F00E5BE124245E5BD2FFF50010E29
:10204E00900000EEF0A3EFF0900072E0B4017EE598
:10205E003445336025AC33AD341DBDFF011C8F02FA
:10206E008E038C068D07903F0F12002EE493FE74A4
:10207E000193FFEFC39AEE9B400280057833124224
:10208E006FAE33AF3474B3BE0025D39F40219000A2
:10209E0000E0FCA3E0FD0FBF00010E903F0F120009
:1020AE002EE493FE740193FFEDC39FEC9E400280DD
:1020BE0005783312003FAE33AF34E56B12424574F0
:1020CE00648E048F05FF1242278D47803390006681
:1020DE00E0602D900000E0FEA3E0FFEFD39400EE51
:1020EE009408400F900066E0B40104C2098002D249
:1020FE0009800D900066E0B40104D2098002C20985
:10210E00900072E064026006900066E0600575BBA8
:10211E00168003754302E543B402028003022212C5
:10212E007E017F00E5BE124245E5BD2FFF50010E38
:10213E00900000EEF0A3EFF0900072E0B4027EE5A6
:10214E003445336025AC33AD341DBDFF011C8F0209
:10215E008E038C068D07903DA512002EE493FE741F
:10216E000193FFEFC39AEE9B400280057833124233
:10217E006FAE33AF3474B3BE0025D39F40219000B1
:10218E0000E0FCA3E0FD0FBF00010E903DA5120084
:10219E002EE493FE740193FFEDC39FEC9E400280EC
:1021AE0005783312003FAE33AF34E56B12424574FF
:1021BE00648E048F05FF1242278D47803390006690
:1021CE00E0602D900000E0FEA3E0FFEFD39400EE60
:1021DE009408400F900066E0B40104C2098002D258
:1021EE0009800D900066E0B40104D2098002C20994
:1021FE00900072E07003754700900066E07002C2B6
:10220E000975BB1FE543B403457E017F00E5BE1291
:10221E004245E5BD2FFF50010E900000EEF0A3EFFA
:10222E00F0740912424574E68E048F05FF124227A0
:10223E008C418D42E54A2DFD50010C74018C068DAA
:10224E00071242378E418F4285424A75BB19E543CC
:10225E00B4040280030224227E017F00E5BE1242F6
:10226E0045E5BD2FFF50010E900000EEF0A3EFF0FC
:10227E0074041242378F4BE565B4010280030223CA
:10228E007D756C00756C00E56CD3940740030223DA
:10229E0034E56C90004112425DE0D3954B501AE547
:1022AE006C90004112425DE0F404254BFEE56C900B
:1022BE00003712425DEEF08017E56C90004112423D
:1022CE005DE0C3954BFEE56C90003712425DEEF07B
:1022DE00E56CC394044009900084E0C3956C503BB8
:1022EE00E56C6029E56C90003712425DFEE0FFEE72
:1022FE0090003FE0D39F4013E56C90003712425D93
:10230E00E090003FF0E56C900040F0800E900037BA
:10231E00E090003FF07400900040F0786C7401265D
:10232E00F64003022295900040E0F4042408F5568E
:10233E00E556D394054006E5B554FDF5B5E558656B
:10234E0056602CE558D394054007E556C3940640D5
:10235E00028005E55104F552855658E556C394049E
:10236E005007E55604F5578003855657755B00E513
:10237E0065D394014061E54BD3946E4004D2118035
:10238E0002C211755605E565B40205A211B34002ED
:10239E008003755607E565B40306A211B3B3400278
:1023AE008003755607E5586556602CE558D394059D
:1023BE004007E556C3940640028005E55104F552E8
:1023CE00855658E556C394045007E55604F55780D4
:1023DE0003855657755B00E55865566008E5510450
:1023EE00F552855658E556B40708E5B54480F5B55F
:1023FE008006E5B5547FF5B5E55664066005E556ED
:10240E00B40808E5B54440F5B58006E5B554BFF50A
:10241E00B575BB13E543B4050280030225367E0174
:10242E007F00E5BE124245E5BD2FFF50010E900024
:10243E0000EEF0A3EFF074041242378F46E564B459
:10244E0002028003022533756C00756C00E56CD3B7
:10245E00940340030224EAE56C90003312425DE0DF
:10246E00D39546501AE56C90003312425DE0F404A9
:10247E002546FEE56C90002D12425DEEF08017E5CC
:10248E006C90003312425DE0C39546FEE56C900001
:10249E002D12425DEEF0E56C6029E56C90002D1278
:1024AE00425DFEE0FFEE900031E0D39F4013E56CFD
:1024BE0090002D12425DE0900031F0E56C900032FC
:1024CE00F0800E90002DE0900031F07400900032FC
:1024DE00F0786C740126F6400302245B900082E0D3
:1024EE007043E52A45296036E559C39403500A9096
:1024FE000032E004C3940340028007900032E004EF
:10250E00F559E559D39402400A900032E004D39471
:10251E000250028007900032E004F55980079000C7
:10252E0032E004F55975BB180543D2ECE55FD39440
:10253E000450030226E975CF01C293AE35AF36744F
:10254E0088D39F74139E4005A2A5B34014AE35AF39
:10255E00367488D39F74139E4005A2A4B3400280A4
:10256E0048783512003FAE35AF36EFB4883BEEB447
:10257E001337A2A5B3500990004FE0D395515002E6
:10258E00800405518011A2A5B3500890004FE0655C
:10259E005160028002D207A2A4B35007E551D39432
:1025AE0001500280041551C207A2A5B3B35006A272
:1025BE00A4B3B340028006753600753500E551654B
:1025CE0052700302268DE55175F040A4FFAEF090D7
:1025DE00032212001EE030E003D38001C3B3400893
:1025EE00E5B54410F5B58006E5B554EFF5B5E55102
:1025FE0075F040A4FFAEF090032312001EE030E011
:10260E0003D38001C3B34008E5B54420F5B5800679
:10261E00E5B554DFF5B5E55175F040A4FFAEF09089
:10262E00032412001EE030E003D38001C39287E53D
:10263E005175F040A4FFAEF090032512001EE0305D
:10264E00E003D38001C3920CE55175F040A4FFAEB8
:10265E00F090032612001EE030E003D38001C392F7
:10266E000DE55175F040A4FFAEF090032712001E49
:10267E00E030E003D38001C3920EC294855152A282
:10268E000740057573CD80037573FFE595C395738C
:10269E004004C2948002D294E54575F00284FF7E18
:1026AE000090018012001EE075F00284FF7E00EFA4
:1026BE0024CDF570E595C395705017A20CB340026A
:1026CE00D291A20DB34002D292A20EB34002D2908A
:1026DE008006C291C292C290022544A210B3500D40
:1026EE00AE25AF2674E8C39F74039E400280057525
:1026FE00FFA0D210AE25AF26EFD39420EE944E500D
:10270E00030227F1120471C28E758D00758B007550
:10271E004C00D28EC2077572007571007573CD753F
:10272E005105752400752300755400755B00C29623
:10273E00900059E06004D2958002C29590004AE064
:10274E00B40104D2978002C297900049E0B401040C
:10275E00D2A08002C2A0A209B34004D2A28002C2BB
:10276E00A290006BE060181238C4A200B34008E5D6
:10277E00B54408F5B58006E5B554F7F5B58002C247
:10278E000090006EE06010123A19A202B34004D21B
:10279E00A18002C2A18002C2A190000E74FDF0A31E
:1027AE0074E8F0E543B40603754300900025E4F0A9
:1027BE00752600752500758D00758B00754C009083
:1027CE000024E0C394035008900024E004F0800637
:1027DE007403900024F0900024E0B40306E5B55491
:1027EE00FEF5B5AE27AF28EFD39410EE9427401C1C
:1027FE00C2CA75CD0075CC00752800752700D2CAE7
:0F280E00754E00752A00752900755500020AE005
:103BCB00000001000132016401960196020002120D
:103BDB0002240200020003000340038003C0040020
:103BEB000440048004C00500060006000600060021
:103BFB00060006000600060000FF01310163019577
:103C0B0001FF01FF0211022302FF02FF02FF033F2C
:103C1B00037F03BF03FF043F047F04BF04FF05FFC3
:103C2B0006FF06FF06FF06FF06FF06FF06FF06FF61
:103C3B000FAA0FA50F9F0F9A0F940F8D0F870F8051
:103C4B000F780F710F680F600F570F4E0F450F3B1B
:103C5B000F300F250F1A0F0E0F020EF50EE80EDBAD
:103C6B000ECC0EBE0EAE0E9F0E8E0E7D0E6C0E5A31
:103C7B000E470E340E200E0C0DF70DE20DCB0DB5CD
:103C8B000D9D0D850D6D0D540D3A0D200D050CE997
:103C9B000CCE0CB10C940C760C580C3A0C1B0BFB89
:103CAB000BDB0BBB0B9A0B790B570B350B130AF179
:103CBB000ACE0AAB0A870A640A400A1C09F809D41F
:103CCB0009B0098C09670943091F08FB08D608B21C
:103CDB00088E086A0846082307FF07DC07B9079612
:103CEB0007730751072F070D06EC06CA06AA0689AC
:103CFB0006690649062A060A05EC05CD05B00592AC
:103D0B0005750558053C0520050504EA04CF04B5E7
:103D1B00049C04820469045104390422040B03F447
:103D2B0003DE03C803B2039D038903750361034DCF
:103D3B00033B03280316030402F202E102D102C083
:103D4B0002B002A00291028202730265025702497D
:103D5B00023C022F02220216020901FD01F201E6CA
:103D6B0001DB01D001C601BB01B101A7019D01948B
:103D7B00018B0182017901700168016001580150CA
:103D8B000148014101390132012B0125011E0118A6
:103D9B000111010B010500FF00FA0FA60FA00F99EF
:103DAB000F920F8B0F840F7C0F740F6B0F620F58DA
:103DBB000F4E0F430F380F2C0F1F0F120F050EF75F
:103DCB000EE80ED80EC80EB70EA50E930E800E6C15
:103DDB000E580E420E2C0E150DFD0DE40DCB0DB134
:103DEB000D950D790D5D0D3F0D200D010CE10CC0F6
:103DFB000C9E0C7C0C590C350C100BEA0BC40B9E57
:103E0B000B760B4F0B260AFD0AD40AAA0A800A5519
:103E1B000A2A09FF09D409A8097C0950092508F9C0
:103E2B0008CD08A10875084A081E07F307C8079DA7
:103E3B0007730749072006F706CE06A6067E065728
:103E4B000630060A05E405BF059B057705540532C8
:103E5B00051004EF04CE04AE048F04710453043533
:103E6B00041903FD03E203C703AD0394037B036350
:103E7B00034B0334031E030802F302DE02CA02B62D
:103E8B0002A30291027F026D025C024C023C022CE7
:103E9B00021D020E020001F201E401D701CA01BEAC
:103EAB0001B101A6019A018F0185017A01700166AA
:103EBB00015D0153014A0141013901310129012100
:103ECB0001190112010B010400FD00F700F000EADB
:103EDB0000E400DE00D900D300CE00C900C400BF4F
:103EEB0000BA00B500B100AD00A800A400A0009C72
:103EFB00009900950091008E008A00870084008154
:043F0B00007E007BB9
:10283E00751A00751900AE19AF1AAC17AD18EDC3A5
:10284E009FEC9E401674FF12421775CF01781A74D2
:10285E000126F6500418E436F650DB22900786E483
:10286E00F0A3F0751000750F00751300751400C2FB
:10287E0012D21322C2AF75D900758F0375B7A57525
:10288E00B7F190F800E4F0758F0175B7A575B7F143
:10289E00E50890F800F075B7A575B7F190F801E46A
:1028AE00F075B7A575B7F190079DE090F802F07539
:1028BE00B7A575B7F19007A1E090F803F075B7A52D
:1028CE0075B7F190079EE090F804F075B7A575B74F
:1028DE00F190079FE090F805F075B7A575B7F190E8
:1028EE0007A0E090F806F075B7A575B7F19007A2AE
:1028FE00E090F807F0758F0075D940D2AF2290079F
:10290E0088E0B4AB61C2AF75D90075B62275F522F9
:10291E00758F0375B7A575B7F1740090F600F07555
:10292E008F01750A00750900AE09AF0A7413BE0057
:10293E00279F402475B7A575B7F190078912001E21
:10294E00E0FC90F60012001EECF0780A740126F6F8
:10295E00500418E436F650D0758F0075F51175B623
:10296E002075D940D2AF22C2AF75D90075F5227548
:10297E000A00750900AE09AF0A7413BE00229F400B
:10298E001F90F60012001EE493FC90078912001EA1
:10299E00ECF0780A740126F6500418E436F650D599
:1029AE0075F51175D940D2AF22900788E0B4AA020E
:1029BE008003022AF4C2AF75D90075B62275F522CE
:1029CE00758F0375B7A575B7F1740090EE00F075AD
:1029DE00B7A575B7F1740090F000F075B7A575B78F
:1029EE00F1740090F200F075B7A575B7F174009010
:1029FE00F400F0758F01750A00750900AE09AF0A73
:102A0E0074FFC39F74019E402475B7A575B7F190EE
:102A1E00004E12001EE0FC90EE0012001EECF0784C
:102A2E000A740126F6500418E436F650CF750A00E3
:102A3E00750900AE09AF0A74FFC39F74019E40244E
:102A4E0075B7A575B7F190024E12001EE0FC90F01E
:102A5E000012001EECF0780A740126F6500418E4F9
:102A6E0036F650CF750A00750900AE09AF0A74FF2D
:102A7E00C39F74019E402475B7A575B7F190044E9F
:102A8E0012001EE0FC90F20012001EECF0780A74A8
:102A9E000126F6500418E436F650CF750A00750973
:102AAE0000AE09AF0A74FFC39F74019E402475B730
:102ABE00A575B7F190064E12001EE0FC90F40012C0
:102ACE00001EECF0780A740126F6500418E436F66F
:102ADE0050CF758F0075F51175B62075D940D2AFF0
:102AEE00743A90074EF022900788E0B4AA02800351
:102AFE00022C32C2AF75D90075B62275F522758FCC
:102B0E000375B7A575B7F1740090E600F075B7A51B
:102B1E0075B7F1740090E800F075B7A575B7F1744C
:102B2E000090EA00F075B7A575B7F1740090EC004F
:102B3E00F0758F01750A00750900AE09AF0A74FFB2
:102B4E00C39F74019E402475B7A575B7F190004ED2
:102B5E0012001EE0FC90E60012001EECF0780A74E3
:102B6E000126F6500418E436F650CF750A007509A2
:102B7E0000AE09AF0A74FFC39F74019E402475B75F
:102B8E00A575B7F190024E12001EE0FC90E80012FF
:102B9E00001EECF0780A740126F6500418E436F69E
:102BAE0050CF750A00750900AE09AF0A74FFC39FB6
:102BBE0074019E402475B7A575B7F190044E1200AE
:102BCE001EE0FC90EA0012001EECF0780A7401265A
:102BDE00F6500418E436F650CF750A00750900AEAB
:102BEE0009AF0A74FFC39F74019E402475B7A57583
:102BFE00B7F190064E12001EE0FC90EC0012001E83
:102C0E00ECF0780A740126F6500418E436F650CF2C
:102C1E00758F0075F51175B62075D940D2AF743A1F
:102C2E0090074EF022900788E0B4AA028003022D8E
:102C3E0070C2AF75D90075B62275F522758F037502
:102C4E00B7A575B7F1740090DE00F075B7A575B72E
:102C5E00F1740090E000F075B7A575B7F1740090AF
:102C6E00E200F075B7A575B7F1740090E400F07549
:102C7E008F01750A00750900AE09AF0A74FFC39F74
:102C8E0074019E402475B7A575B7F190004E1200E1
:102C9E001EE0FC90DE0012001EECF0780A74012695
:102CAE00F6500418E436F650CF750A00750900AEDA
:102CBE0009AF0A74FFC39F74019E402475B7A575B2
:102CCE00B7F190024E12001EE0FC90E00012001EC2
:102CDE00ECF0780A740126F6500418E436F650CF5C
:102CEE00750A00750900AE09AF0A74FFC39F74011F
:102CFE009E402475B7A575B7F190044E12001EE0E4
:102D0E00FC90E20012001EECF0780A740126F650D8
:102D1E000418E436F650CF750A00750900AE09AFF7
:102D2E000A74FFC39F74019E402475B7A575B7F151
:102D3E0090064E12001EE0FC90E40012001EECF015
:102D4E00780A740126F6500418E436F650CF758FC3
:102D5E000075F51175B62075D940D2AF743A90074B
:102D6E004EF022900788E0B4AA028003022EAEC273
:102D7E00AF75D90075B62275F522758F0375B7A597
:102D8E0075B7F1740090D600F075B7A575B7F174EC
:102D9E000090D800F075B7A575B7F1740090DA0001
:102DAE00F075B7A575B7F1740090DC00F0758F0162
:102DBE00750A00750900AE09AF0A74FFC39F74014E
:102DCE009E402475B7A575B7F190004E12001EE017
:102DDE00FC90D60012001EECF0780A740126F65014
:102DEE000418E436F650CF750A00750900AE09AF27
:102DFE000A74FFC39F74019E402475B7A575B7F181
:102E0E0090024E12001EE0FC90D80012001EECF054
:102E1E00780A740126F6500418E436F650CF750A77
:102E2E0000750900AE09AF0A74FFC39F74019E407E
:102E3E002475B7A575B7F190044E12001EE0FC90F4
:102E4E00DA0012001EECF0780A740126F65004180F
:102E5E00E436F650CF750A00750900AE09AF0A7454
:102E6E00FFC39F74019E402475B7A575B7F19006F8
:102E7E004E12001EE0FC90DC0012001EECF0780AF0
:102E8E00740126F6500418E436F650CF758F00758F
:102E9E00F51175B62075D940D2AF743A90074EF041
:102EAE0022C2AF75D90075F522750A00750900AEFC
:102EBE0009AF0A74FFC39F74019E401F90EE00126B
:102ECE00001EE493FC90004E12001EECF0780A7483
:102EDE000126F6500418E436F650D4750A0075092A
:102EEE0000AE09AF0A74FFC39F74019E401F90F09D
:102EFE000012001EE493FC90024E12001EECF078BD
:102F0E000A740126F6500418E436F650D4750A00F9
:102F1E00750900AE09AF0A74FFC39F74019E401F6E
:102F2E0090F20012001EE493FC90044E12001EEC70
:102F3E00F0780A740126F6500418E436F650D4756B
:102F4E000A00750900AE09AF0A74FFC39F74019E93
:102F5E00401F90F40012001EE493FC90064E1200E7
:102F6E001EECF0780A740126F6500418E436F6507A
:102F7E00D475F51175D940D2AF22C2AF75D900758F
:102F8E00F522750A00750900AE09AF0A74FFC39FDA
:102F9E0074019E401F90E60012001EE493FC900008
:102FAE004E12001EECF0780A740126F6500418E456
:102FBE0036F650D4750A00750900AE09AF0A74FFD3
:102FCE00C39F74019E401F90E80012001EE493FC04
:102FDE0090024E12001EECF0780A740126F6500490
:102FEE0018E436F650D4750A00750900AE09AF0A1A
:102FFE0074FFC39F74019E401F90EA0012001EE4EE
:10300E0093FC90044E12001EECF0780A740126F622
:10301E00500418E436F650D4750A00750900AE094E
:10302E00AF0A74FFC39F74019E401F90EC00120004
:10303E001EE493FC90064E12001EECF0780A74010A
:10304E0026F6500418E436F650D475F51175D940AD
:10305E00D2AF22C2AF75D90075F522750A00750977
:10306E0000AE09AF0A74FFC39F74019E401F90DE2D
:10307E000012001EE493FC90004E12001EECF0783D
:10308E000A740126F6500418E436F650D4750A0078
:10309E00750900AE09AF0A74FFC39F74019E401FED
:1030AE0090E00012001EE493FC90024E12001EEC03
:1030BE00F0780A740126F6500418E436F650D475EA
:1030CE000A00750900AE09AF0A74FFC39F74019E12
:1030DE00401F90E20012001EE493FC90044E12007A
:1030EE001EECF0780A740126F6500418E436F650F9
:1030FE00D4750A00750900AE09AF0A74FFC39F7438
:10310E00019E401F90E40012001EE493FC90064EB8
:10311E0012001EECF0780A740126F6500418E436FC
:10312E00F650D475F51175D940D2AF22C2AF75D90C
:10313E000075F522750A00750900AE09AF0A74FF15
:10314E00C39F74019E401F90D60012001EE493FC94
:10315E0090004E12001EECF0780A740126F6500410
:10316E0018E436F650D4750A00750900AE09AF0A98
:10317E0074FFC39F74019E401F90D80012001EE47E
:10318E0093FC90024E12001EECF0780A740126F6A3
:10319E00500418E436F650D4750A00750900AE09CD
:1031AE00AF0A74FFC39F74019E401F90DA00120095
:1031BE001EE493FC90044E12001EECF0780A74018B
:1031CE0026F6500418E436F650D4750A0075090038
:1031DE00AE09AF0A74FFC39F74019E401F90DC00BE
:1031EE0012001EE493FC90064E12001EECF0780ABC
:1031FE00740126F6500418E436F650D475F51175A0
:10320E00D940D2AF22E51464046006E59964FF60EC
:10321E00028031A2124004D2128027E51460087495
:10322E00E62514900023F0E513600874F025139042
:10323E000023F0E514B4010280FE7514007513002E
:10324E00C2128002C212E514903B6EF828287375E4
:10325E001400E599B4FF03751301E599B4FE0375E7
:10326E001302E599B4FD03751303E599B4FC0375D8
:10327E001304E599B4FA03751305E599B4FB0675C5
:10328E001401120471E599B4F9067514041204714F
:10329E00E599D394E54007E599C394F04002801672
:1032AE008599157514027E017F00E515C394E6120B
:1032BE0042458E0D8F0E900786E4F0A3F0E599D36C
:1032CE0094C44007E599C394E64002802885991579
:1032DE0075140374E5C39515F50E750D00AE0DAF9F
:1032EE000E903BCB12002EE493F874019390078658
:1032FE00C8F0A3C8F0D299023782900786E0FEA3E9
:10330E00E0FFEFC39400EE94054009EFD394FFEE77
:10331E0094064013900786E0FEA3E0FF90004E1245
:10332E00001EE599F0800385996D90078612000EB8
:10333E00900786E0FEA3E0FFEFB40106EEB40702AD
:10334E00800302359290074EE0B43C0280030235B2
:10335E0092A20AB35005A20BB34003023485C29C5D
:10336E0090007AE090078CF0900057E090078DF077
:10337E00900062E090078EF0900063E090078FF06F
:10338E00900074E0900790F090007CE0900791F030
:10339E0090007DE0900792F0900080E0900793F00F
:1033AE00900081E0900794F090013AE0900795F03C
:1033BE0090013BE0900796F090013CE0900797F06B
:1033CE00900090E0900798F0900091E0900799F0AF
:1033DE00900092E090079AF0900093E090079BF097
:1033EE00900094E090079CF0900095E090079DF07F
:1033FE00900096E090079EF0900097E090079FF067
:10340E00900099E09007A0F090009AE09007A1F04C
:10341E0090009BE09007A2F090009CE09007A3F034
:10342E007400900082F012008F74AB900788F01237
:0A343E00290C74AA900788F0E559E4
:063B6E0002325D02330883
:10344800903B8FF828287380121229B7800D122A12
:0B345800F58008122C338003122D7148
:0F3B8F0002344F02345102345602345B02346068
:10346300900788E4F090013AE0700C90013BE07023
:103473000690013CE060028004C20A8002D20A0284
:103483003587C29C900078E0900789F090005EE059
:1034930090078AF090005FE090078BF090007AE04D
:1034A30090078CF0900057E090078DF0900062E059
:1034B30090078EF0900063E090078FF0900074E027
:1034C300900790F090007CE0900791F090007DE0F1
:1034D300900792F0900080E0900793F0900081E0D5
:1034E300900794F090013AE0900795F090013BE04B
:1034F300900796F090013CE0900797F0900090E0E1
:10350300900798F0900091E0900799F0900092E076
:1035130090079AF0900093E090079BF0900094E05E
:1035230090079CF0900095E090079DF0900096E046
:1035330090079EF0900097E090079FF0900099E02D
:103543009007A0F090009AE09007A1F090009BE014
:103553009007A2F090009CE09007A3F07400900005
:1035630082F074AB900788F012290C74AA90078834
:10357300F01229B7122AF5122C33122D71D29C7531
:1035830099FB80FED29C7514007513007599FB029C
:103593003782900786E0FEA3E0FFEF4E7006859921
:1035A30010750F00900786E0FEA3E0FF74016F4ED5
:1035B300701BAC0FAD10AA0DAB0EED2BFBEC3AFA62
:1035C3008A068B0790004E12001EE599F09007863D
:1035D30012000E900786E0FEA3E0FF74026F4E70A8
:1035E3000C12008F8515997514007513000237822C
:1035F300900786E0FEA3E0FF90004E12001EE599BF
:10360300F090078612000E900786E0FEA3E0FFAC61
:103613000DAD0E8F028E038C068D07903C031200B6
:103623002EE493F9740193FEEAD39EEB9940098546
:103633001599751400751300023782900786E0FE12
:10364300A3E0FF90004E12001EE599F0900786124A
:10365300000E900786E0FEA3E0FFEFB40006EEB491
:103663000102800302378290001CE0D394C7400B11
:1036730090001CE0C394C8F516801A90001CE0D398
:103683009463400B90001CE0C39464F5168006908D
:10369300001CE0F516E51675F002A4FFAEF08F6C82
:1036A300EF90004E12425DEFFCE0FDEC90005112F2
:1036B300425DEDFCE0FDEC2DB5160280030237748C
:1036C3000FEF90004E12425DE56CFFE0FCEF9000BF
:1036D3005212425DECFFE0FCEFC39CB5160280037F
:1036E300023774E56C90005012425DE56CFFE0FC1C
:1036F300EF90005312425DECFFE0FCEF2CB5167126
:10370300E56C90005412425DE0C3951690079DF05E
:10371300E56C90005512425DE0C3951690079EF04C
:10372300E56C90005812425DE0C3951690079FF038
:10373300E56C90005912425DE0C395169007A0F026
:10374300E56C90005A12425DE0C395169007A1F014
:10375300E56C90005B12425DE0C395169007A2F002
:103763001228827599F975186475170012283E801E
:0F377300FE7599FF75186475170012283E80FEC9
:093B74000235950235F302363EDC
:1037820022E513903B7DF82828730238C390078600
:10379200E0FEA3E0FF90001212001EE0F5999007F0
:1037A2008612000E900786E0FEA3E0FF74116F4EB2
:1037B20070037513000238C38563990238C39007FA
:1037C20086E0FEA3E0FF90004E12001EE0F599EFA6
:1037D200B40107EEB4070375130090078612000EBA
:0737E2000238C3900787E0E5
:0F3B7D0002378C02378F0237BA0237C00237E5A2
:1037E900903B9EF82828738524990238B8852A9930
:1037F9000238B88544990238B88547990238B8859E
:1038090051990238B88561990238B88556990238B4
:10381900B88559990238B8756F00900069E070064B
:10382900900068E060028016A2A44006E56F440497
:10383900F56FA2A54006E56F4402F56F801A900066
:103849004AE0B40106E56F4410F56F900049E0B411
:103859000106E56F4420F56FA207B34006E56F4402
:1038690001F56FA209B34006E56F4408F56F856F4E
:1038790099803CA213B340077599FAC2138017A225
:103889000FB3400575990F800B900023E0F59990CF
:103899000023E4F0C20F80178542998012854B9965
:0F38A900800D85469980087599FC800375130082
:103B9E000237F00237F60237FC023802023808020A
:103BAE00380E02381402381A02382002387C0238D5
:0D3BBE00A10238A60238AB0238B00238B5BB
:0B38B80090078612000E8003120048EB
:033B8C000238C03C
:1038C3002290006BE0B4010385241190006BE0B4F7
:1038D3000203852A1190006BE0B403038544119021
:1038E300006BE0B4040385471190006BE0B405035B
:1038F30085511190006BE0B4060385561190006B5F
:10390300E0B4070385591190006CE0FE90006DE070
:10391300C39E500302399A90006BE0D39404402C69
:1039230090006CE0D39511500990006DE0C39511A0
:1039330050028002D20090006CE0D39511500990A0
:10394300006DE0C395115002C200804990006BE006
:10395300B4041890006DE0C395115002D20090009A
:103963006CE0D395114002C200802A90006CE0C342
:103973009511500990006DE0D3951150028002D249
:103983000090006CE0D39511500990006DE0C39551
:10399300115002C200807E90006BE0D39404402C4F
:1039A30090006CE0C39511400990006DE0D3951130
:1039B30040028002C20090006CE0C3951140099060
:1039C300006DE0D395114002D200804990006BE076
:1039D300B4041890006CE0C395115002C20090002B
:1039E3006DE0D395114002D200802A90006CE0C3B1
:1039F3009511400990006DE0D395114002D20090DB
:103A0300006CE0D39511400990006DE0C39511401F
:103A1300028002C2002290006EE0B40103852411EB
:103A230090006EE0B40203852A1190006EE0B403A7
:103A33000385441190006EE0B404038547119000A0
:103A43006EE0B4050385511190006EE0B406038562
:103A5300561190006EE0B4070385591190006FE092
:103A6300FE900070E0C39E5003023AEF90006EE0B8
:103A7300D39404402C90006FE0D39511500990002B
:103A830070E0C3951150028002D20290006FE0D320
:103A930095115009900070E0C395115002C2028045
:103AA3004990006EE0B40418900070E0C395115083
:103AB30002D20290006FE0D395114002C202802A25
:103AC30090006FE0C395115009900070E0D39511F9
:103AD30050028002D20290006FE0D39511500990FA
:103AE3000070E0C395115002C202807E90006EE028
:103AF300D39404402C90006FE0C3951140099000CB
:103B030070E0D3951140028002C20290006FE0C3BF
:103B130095114009900070E0D395114002D20280C4
:103B23004990006EE0B4041890006FE0C395115003
:103B330002C202900070E0D395114002D202802AA3
:103B430090006FE0C395114009900070E0D3951188
:103B53004002D20290006FE0D395114009900070AB
:0B3B6300E0C3951140028002C2022264
:09425D002582F58250020583223E
:10002E00EF2F500205832582F582E5833E2EF58360
:01003E00229F
:08000300C3EF9DFFEE9CFE22FD
:08003F000806B60002180622B3
:0D000E00A3E004F07006124253E004F0225B
:08426F000816B6FF0218162222
:0E423700048007C3CE13CECF13CFD5E0F622FE
:1040E500BC000FBE0008ED8FF084FFADF022E4FEAA
:1040F500FF22BE000DEF60FE54F0606F20E7030263
:10410500419BEAC0E0EBC0E078017A0075F001EE72
:1041150020E710EF25E0FFEE33FE0AC5F023C5F0DA
:1041250030E7F0EA5407F9096A7A007B0060010874
:10413500C3EC9E40167004ED9F4010ED9FFDEC9E74
:10414500FCE5F0CA4ACA03F5F08005E5F003F5F091
:10415500C3EE13FEEF13FFD9D77908CACBCAD8D05F
:10416500EAFEEBFFD0E0FBD0E0FA22EC8FF084FC16
:10417500ED54F045F0C48FF084FEEDC454F045F0E5
:10418500C48FF084FDEEC4FE54F02DFFEE540F3CB9
:10419500FEADF07C0022790078008FF0EC7E0820DF
:1041A500E70DC3CD33CD33C933C9C833C8DEF08479
:1041B50049F9E5F08FF0BE00E6FD7C00E9FFE8FE79
:0141C50022D7
:0E424500F88FF0A4FFE5F0CE88F0A42EFE2244
:10421700600D782B024221007830D8FED5E0F822D5
:10422700EEC0E07E001240E5EFFDEEFCD0E0FE229E
:03000B000241C6E9
:03001B000241E1BE
:03002B000241FC93
:0300000002426653
:0942660075817475D00002065840
:0B001E00E5822FF582E5833EF583228A
:0A4253000582D58202158315822230
:1041C600C0E0C0F0C083C082C0D075D00012064DDA
:1041D600D0D0D082D083D0F0D0E032C0E0C0F0C0E2
:1041E60083C082C0D075D000120650D0D0D082D005
:1041F60083D0F0D0E032C0E0C0F0C083C082C0D02F
:1042060075D000120653D0D0D082D083D0F0D0E043
:014216003275
:00000001FF
